S0220000687474703A2F2F737265636F72642E736F75726365666F7267652E6E65742F1D
S12300000C9438000C9481160C94361E0C945F000C945F000C945F000C945F000C945F00DE
S12300200C945F000C94F91E0C945F000C94FD220C945F000C9462170C943C170C94121675
S12300400C94FD230C945F000C947C230C945F000C94A2240C946A240C945F000C945F000D
S12300600C945F000C945F000C945F000C945F0011241FBECFEFD0E1DEBFCDBF14BEA895C7
S123008088E10FB6F89480936000109260000FBE15E0A0E0B1E0EEEBFCE402C005900D92AB
S12300A0AC31B107D9F716E0ACE1B5E001C01D92AA3CB107E1F70E94750E0C945E260C94F0
S12300C0000020E030E0D901AC54BF4F0E944026802DF901EF5BFE4F80832F5F3F4F203A65
S12300E0310589F720E030E0D901A857BE4F0E944026802DF901E65CFE4F80832F5F3F4FF3
S12301002530310589F712BC11BC089520E030E0F901EF5BFE4F8081D901AC54BF4F082ED8
S12301200E944D262F5F3F4F203A310589F712BC11BC08954E9B11C020E030E0D9015096B8
S12301400E944026802DF901EF51FE4F80832F5F3F4F203A310591F0F1CF20E030E0D90185
S1230160A859BD4F0E944026802DF901EF51FE4F80832F5F3F4F203A310589F712BC11BC68
S123018008954E9B11C020E030E0F901EF51FE4F8081D9015096082E0E944D262F5F3F4F45
S12301A0203A310591F0F1CF20E030E0F901EF51FE4F8081D901A859BD4F082E0E944D26A0
S12301C02F5F3F4F203A310589F712BC11BC089520E931E0D9010E944026802D2055314028
S12301E0F901EF57FD4F80832F5A3E4F81E0203F380781F712BC11BC089520E430E0F90199
S1230200EF57FD4F8081D901A05BBE4F082E0E944D262F5F3F4F203A310589F712BC11BC53
S12302200895A2E0B0E00E944026802D90E090931F0180931E0120911E0130911F01A3E03D
S1230240B0E00E944026802D90E0982F8827820F931F90931F0180931E01A4E0B0E00E9401
S12302604026802D90E090932101809320012091200130912101A5E0B0E00E944026802DFF
S123028090E0982F8827820F931F9093210180932001A6E0B0E00E944026802D90E090935A
S12302A00101809300012091000130910101A7E0B0E00E944026802D90E0982F8827820F6C
S12302C0931F9093010180930001A1E0B0E00E944026802D80931C05A8E0B0E00E94402615
S12302E0802D80931301A9E5B1E00E944026802D80932A01A2E0B4E00E944026902D892F81
S12303008150843078F080912A01843039F481E08093180183E68093CF0506C082E08093B7
S1230320180102C090931801A9E0B0E00E944026802D80931201AEE0B0E00E944026802DDB
S123034080932301ABE0B0E00E944026802D80931901ACE0B0E00E944026802D80931A0166
S1230360AFE6B1E00E944026802D80931B01A2EFB1E00E944026802D80938A0580918A0556
S1230380882319F081E080938A05ADE0B0E00E944026802D26E0829FC0011124909315017A
S12303A080931401A1E7B1E00E944026802D8093F305A0E7B1E00E944026802D8093F10562
S12303C08AE08093240681E080932206AFE8B1E00E944026802D80932B0180912B0181FFFD
S12303E005C080912B01827F80932B0180912B0185FF05C080912B018F7280932B01A4EF21
S1230400B1E00E944026802D24E1829FC00111249093C8058093C705A5EFB1E00E9440267A
S1230420802D8093C405A6EFB1E00E944026802D8093C205A7EFB1E00E944026802D80938B
S1230440C105A8EFB1E00E944026802D90E09093C0058093BF052091BF053091C005A9EF33
S1230460B1E00E944026802D90E0982F8827820F931F9093C0058093BF05ABEFB1E00E947D
S12304804026802D90E090932F0180932E0120912E0130912F01ACEFB1E00E944026802D8E
S12304A090E0982F8827820F931F90932F0180932E01ADEFB1E00E944026802D90E0909305
S12304C03101809330012091300130913101AEEFB1E00E944026802D90E0982F8827820F73
S12304E0931F9093310180933001AFEFB1E00E944026802D90E0909333018093320120910B
S1230500320130913301A0E0B2E00E944026802D90E0982F8827820F931F90933301809355
S1230520320120E030E0D901A25ABE4F0E944026802DF901EF5DFC4F8083D901AE58BE4F5B
S12305400E944026802DF901E053FA4F8083D901A458BE4F0E944026802D808B2F5F3F4FAA
S12305602A30310501F7A7E0B2E00E944026802D80933601A3E0B2E00E944026802D8093FA
S1230580370120E030E0F901EF5FF94F84E6808BD901A45EBD4F0E944026802D80832F5FDC
S12305A03F4F2031310579F720E030E0D901A759BE4F0E944026802DF901EB5DFE4F808374
S12305C02F5F3F4F2430310589F720E030E0D901A25DBD4F0E944026802DF901EF50FB4FC4
S12305E080832F5F3F4F2031310589F7ADE6B1E00E944026802D80932201A1EFB1E00E94FF
S12306004026802D80938905A0EFB1E00E944026802D80932901A6E0B2E00E944026802D43
S12306208093240120E030E0D901AA54BC4F0E944026802DF901E55DFC4F80832F5F3F4F30
S12306402031310589F7A7ECB3E00E944026802D80933801A8ECB3E00E944026802D809379
S12306603901A4EDB3E00E944026802D80939105A5EDB3E00E944026802D80939205A6EDA3
S1230680B3E00E944026802D80939305A7EDB3E00E944026802D80939405A8EEB3E00E9410
S12306A04026802D90E090932D0180932C0120912C0130912D01A9EEB3E00E944026802D76
S12306C090E0982F8827820F931F90932D0180932C01AAEEB3E00E944026802D80938C05D8
S12306E012BC11BC089580911E0190911F01A2E0B0E0082E0E944D2680911E0190911F017F
S1230700892F9927A3E0B0E0082E0E944D268091200190912101A4E0B0E0082E0E944D262B
S12307208091200190912101892F9927A5E0B0E0082E0E944D268091000190910101A6E0AD
S1230740B0E0082E0E944D268091000190910101892F9927A7E0B0E0082E0E944D2680919A
S12307601301A8E0B0E0082E0E944D2680911201A9E0B0E0082E0E944D2612BC11BC08953E
S123078080E0A1EFB1E0082E0E944D268AE0A0EFB1E0082E0E944D2680918A05A2EFB1E0F2
S12307A0082E0E944D2684E0A9E5B1E0082E0E944D2685E0ACE0B0E0082E0E944D2682E3EB
S12307C0AFE6B1E0082E0E944D2624E1A1E7B1E0022E0E944D2691E0A0E7B1E0092E0E94DF
S12307E04D2688ECA4EFB1E0082E0E944D26A5EFB1E0092E0E944D26A6EFB1E0022E0E9436
S12308004D268AE5A7EFB1E0082E0E944D2688EEA8EFB1E0082E0E944D2683E0A9EFB1E00B
S1230820082E0E944D2680912E0190912F01ABEFB1E0082E0E944D2680912E0190912F01D1
S1230840892F9927ACEFB1E0082E0E944D268091300190913101ADEFB1E0082E0E944D2698
S12308608091300190913101892F9927AEEFB1E0082E0E944D268091320190913301AFEFB7
S1230880B1E0082E0E944D268091320190913301892F9927A0E0B2E0082E0E944D268CED91
S12308A0A7E0B2E0082E0E944D2686EEA3E0B2E0082E0E944D262CE132E088ECD901082E59
S12308C00E944D262F5F3F4F82E02C323807A9F782E2AFE8B1E0082E0E944D2681E0A6E086
S12308E0B2E0082E0E944D2612BC11BC0895CF92DF92EF92FF920F931F93CF93DF93C0E033
S1230900D0E0A5E0B2E00E944026202D30E040E050E0A3EDB3E00E944026602D6E01CC0C58
S1230920DD1C8BE393E0C80ED91EF601E080F18070E080E090E00E94B12500E010E0A80133
S123094097010E94B12524E630E040E050E00E94032679018A01CA01B90124EF31E040E080
S123096050E00E94B12528EC30E040E050E0E20EF31E041F151FA80197010E940326CA0128
S1230980B9012FEF30E040E050E00E94B12525E030E040E050E00E94032682E0220F331F8E
S12309A0441F551F8A95D1F7CA01B90124E630E040E050E00E940326F601318320832196B6
S12309C0C732D10509F09DCFC0E0D0E0A9ECB3E00E944026202D30E040E050E0A3EDB3E08F
S12309E00E944026602D6E01CC0CDD1C89E893E0C80ED91EF601E080F18070E080E090E085
S1230A000E94B12500E010E0A80197010E94B12524E630E040E050E00E94032679018A0197
S1230A20CA01B90124EF31E040E050E00E94B12528EC30E040E050E0E20EF31E041F151F75
S1230A40A80197010E940326CA01B9012FEF30E040E050E00E94B12525E030E040E050E0A6
S1230A600E94032612E0220F331F441F551F1A95D1F7CA01B90124E630E040E050E00E9453
S1230A800326F601318320832196C732D10509F09DCFC0E0D0E0AAECB3E00E944026202D22
S1230AA030E040E050E0A3EDB3E00E944026602D6E01CC0CDD1C87ED93E0C80ED91EF6012F
S1230AC0E080F18070E080E090E00E94B12500E010E0A80197010E94B12524E630E040E0E6
S1230AE050E00E94032679018A01CA01B90124EF31E040E050E00E94B12528EC30E040E03D
S1230B0050E0E20EF31E041F151FA80197010E940326CA01B9012FEF30E040E050E00E9498
S1230B20B12525E030E040E050E00E940326A2E0220F331F441F551FAA95D1F7CA01B90143
S1230B4024E630E040E050E00E940326F601318320832196C732D10509F09DCFC0E0D0E0D3
S1230B60A4E0B2E00E944026202D30E040E050E0A3EDB3E00E944026602D6E01CC0CDD1CAE
S1230B8085E294E0C80ED91EF601E080F18070E080E090E00E94B12500E010E0A801970138
S1230BA00E94B12524E630E040E050E00E94032679018A01CA01B90124EF31E040E050E086
S1230BC00E94B12528EC30E040E050E0E20EF31E041F151FA80197010E940326CA01B9013C
S1230BE02FEF30E040E050E00E94B12525E030E040E050E00E940326E2E0220F331F441F23
S1230C00551FEA95D1F7CA01B90124E630E040E050E00E940326F601318320832196C7325D
S1230C20D10509F09DCFDF91CF911F910F91FF90EF90DF90CF900895EAE7F0E01082109207
S1230C407C0080E880BF87EE808311B888E790E090931F0580931E0508950F931F93CF937D
S1230C60DF93282F30E0F901EE0FFF1FEE5FFE4F0081118143E0033F140718F0E2E3F0E0B8
S1230C804CC053E00F3D150718F0EAE0F0E045C0C0E0D0E087E290E0A901489F9001499FCF
S1230CA0300D589F300D1124D901AC0FBD1FAA0FBB1FA55CBC4F8D919C9111978017910758
S1230CC030F5FE013197E20FF31FEE0FFF1FE55CFC4F20813181608171814D915C91FE018A
S1230CE0EE0FFF1FEE0FFF1FEC0FFD1F3596201B310BC901880F991F880F991F641B750BFA
S1230D00820F931F0E94DC25E60FF71F06C02196C732D10549F6E8ECF0E0CF01DF91CF910F
S1230D201F910F9108959C0180911C0584FF1BC022533040C901E3E0880F991FEA95E1F77D
S1230D40220F331F280F391F2455354F442737FD4095542F60E579E784E090E00E94252623
S1230D60822F90E0089580911C0585FD03C084E690E0089522533040C90163E0880F991F82
S1230D806A95E1F7220F331F280F391F2455354F442737FD4095542F60E579E784E090E0F9
S1230DA00E9425262C592695822F90E008950F931F93CF93DF93AC01E0E0F0E0EF01CC0F14
S1230DC0DD1FDE01AD58BB4F8D919C91119748175907C0F56D917C913197EE0FFF1FDF01F0
S1230DE0AD58BB4F8D919C911197681B790B8D919C91C557DB4F28813981E557FB4F0081EB
S1230E001181481B590B84E690E0DC014A9FC0014B9F900D5A9F900D11240E94DC25201BE4
S1230E20310B0190F081E02D629FC001639F900D729F900D112464E670E00E94DC256E0F65
S1230E407F1F09C03196EA30F10509F0B7CF60919F047091A004CB01DF91CF911F910F91AC
S1230E6008950F931F93CF93DF93AC018091B3049091B4044817590718F4E0EFF0E057C0DA
S1230E808091CF049091D0048417950718F4E0E0F0E04DC0E1E0F0E0EF01CC0FDD1FDE015E
S1230EA0AD54BB4F8D919C91119748175907C0F56D917C913197EE0FFF1FDF01AD54BB4FE3
S1230EC08D919C911197681B790B8D919C91EF52FB4F20813181CF52DB4F08811981481B1A
S1230EE0590B84E690E0DC014A9FC0014B9F900D5A9F900D11240E94DC25201B310B01902C
S1230F00F081E02D629FC001639F900D729F900D112464E670E00E94DC25E61BF70B07C004
S1230F203196EE30F10509F0B7CFEEEFF0E0CF01DF91CF911F910F91089580911E019091C8
S1230F401F0190931D0180931C018091920520912E0530912F0590E08F5B9F4F8217930700
S1230F605CF480919205882339F080917D0590917E0550E041E013C08091920520912E05BA
S1230F8030912F0590E0C2968217930734F480919205882311F051E001C050E040E080918E
S1230FA09105209134053091350590E0C2968217930774F480919105882351F084EC99E0D3
S1230FC090931D0180931C0180917D0590917E0580919305209132053091330590E0C29613
S1230FE08217930754F480919305882331F084EC99E090931D0180931C0180919405209148
S123100030053091310590E0C2968217930754F480919405882331F084EC99E090931D01BD
S123102080931C01442311F086E903C0552321F082E3809379050895109279050895A895CC
S123104082E50E94F72483E10E94F72480917D0590917E05892F99270E94F72480917D0548
S123106090917E050E94F72480913405909135050E94F72480912E0590912F050E94F72453
S123108080911E0590911F050E94F72480912C0590912D050E94F72480912A0590912B0533
S12310A00E94F72480912605909127050E94F72480918305909184056091180170E00E94EA
S12310C0DC25CB010E94F724809182050E94F724809181050E94F7242091FF05309100065D
S12310E08091CB059091CC05E3E096958795EA95E1F78170232F3327822B0E94F7248091A0
S1231100FF05909100060E94F7248091F8059091F9050E94F72480919B050E94F72480917A
S12311202405909125050E94F7248091CD059091CE05969587950E94F72489B1869586952F
S1231140817090E0909337058093360583B18695817090E090933905809338058091010505
S12311609091020590933B0580933A058091F4059091F50590933D0580933C0520919A0560
S123118030E0220F331FF901E25DFA4F80819181892F990F990B93E0220F331F9A95E1F722
S12311A0822B0E94F724E0919A05F0E0EE0FFF1FE25DFA4F808191810E94F7248DEA0E9455
S12311C0F72480919A058F5F80939A05883010F010929A050895CF92DF92EF92FF920F9384
S12311E01F93CF93DF93A89588E10FB6F89480936000109260000FBE0E944325882309F47A
S12312006AC50E94D42490939905809398058236910509F4E8C28336910508F041C080359E
S1231220910509F45AC381359105E8F48534910509F4D1C08634910568F48932910509F4FB
S12312409DC48134910509F48DC08832910509F040C571C48634910509F446C18D34910566
S123126009F037C5BDC18535910509F4EAC38635910548F48235910509F4ABC3833591056A
S123128009F027C5CDC48835910509F422C48136910509F442C08735910509F01AC594C3D1
S12312A08936910509F4CAC28A369105C8F48536910509F408C28636910548F48336910545
S12312C009F494C28436910509F003C504C58636910509F4E7C08736910509F0FAC4D5C246
S12312E08037910509F4FEC28137910548F48D36910509F434C18F36910509F0EAC401C444
S12313008937910509F45DC48A37910509F471C28837910509F0DDC46CC281E60E94F7248D
S123132080EA0E94F72410929905109298050EC0EF5BFE4F80810E94F72480919805909111
S1231340990501969093990580939805E0919805F0919905E03AF10558F382E30E944824E8
S12313608EE9B7C41092990510929805C0E0D0E00E944325882341F1C0919805D0919905D4
S1231380C03AD10589F40E94D42490939905809398058E3B910519F4C6E1DAEF15C080912F
S12313A098050E94F724FBCF0E94D424CF5BDE4F8883809198059091990501969093990544
S12313C080939805C0E0D0E021964AEFC030D40708F081C4CDCFC0E0D0E00E944325882370
S12313E009F459C00E94D4248A3B910509F073C488E10FB6F89480936000109260000FBEB2
S123140010929905109298053EC0885B0E94F7248DEF0E94F72420919805309199058AEF4C
S123142090E0289FE001299FD00D389FD00D112407C0DE010E944026802D0E94F724219633
S123144020919805309199052F5F3F4F8AEF90E0AC01249FC001259F900D349F900D11249F
S123146021503040C817D90720F3822F885B80950E94F72480919805909199050196909328
S123148099058093980580919805909199058430910508F4BACF21965AEFC030D50708F0FA
S12314A01AC49BCF86E60E94F72480EA0E94F72410929905109298050EC0EF51FE4F8081B5
S12314C00E94F724809198059091990501969093990580939805E0919805F0919905E03A8F
S12314E0F10558F389E9F5C3109299051092980500E010E00E944325882349F1C091980551
S1231500D0919905C03AD10591F40E94D4249093990580939805893B910519F406E11AEF11
S123152016C0E0919605F0919705099510C00E94D424CF51DE4F88838091980590919905DB
S12315400196909399058093980500E010E00F5F1F4F8AEF0030180708F0BDC3CBCF8DE686
S12315600E94F72489E00E94F72480911E0190911F010E94F72480911E0190911F01892F2D
S123158099270E94F72480912001909121010E94F7248091200190912101892F99270E9409
S12315A0F72480910001909101010E94F7248091000190910101892F99270E94F72480919F
S12315C013010E94F724809112010E94F724AAE0B0E00E944026802D0E94F72482E979C322
S12315E01092990510929805C0E0D0E00E9443258A3008F461C00E94D42490931F01809347
S12316001E0100911E0110911F010E94D424982F8827800F911F90931F0180931E010E94D0
S1231620D424909321018093200100912001109121010E94D424982F8827800F911F90934E
S12316402101809320010E94D424909301018093000100910001109101010E94D424982FC7
S12316608827800F911F90930101809300010E94D424809313010E94D424809312010E941C
S1231680D424AAE0B0E0082E0E944D260E94AE1E0E94D424823B910551F40E947303E091C0
S12316A09605F09197050995CFE6DAEF05C0E0919605F0919705099521964AEFC030D4070B
S12316C008F009C393CF85E60E94F72483E10E94F72410929905109298050EC0EF5DFC4FB3
S12316E080810E94F724809198059091990501969093990580939805E0919805F091990586
S1231700EA30F10558F3809119010E94F72480911A010E94F72483E00E94492480912501F0
S12317200E94F724809126010E94F724809127010E94F724809128010E94F72480911401E0
S12317409091150166E070E00E94DC25CB010E94F724809122010E94F724AEE6B1E00E94D4
S12317604026802D0E94F7248AE90E94F7248CE60E94F72484E10E94F72410929905109232
S123178098050EC0E053FA4F80810E94F7248091980590919905019690939905809398052B
S12317A0E0919805F0919905EA30F10558F310929905109298050EC0E053FA4F80890E9429
S12317C0F724809198059091990501969093990580939805E0919805F0919905EA30F10538
S12317E058F383E976C20E94860075C20E94C10072C20E941F086FC20E94D424C82FD0E0C5
S12318000E94D424C817D90709F065C20E94D4248C0190939905809398050E94D4240817FA
S1231820190709F058C20E94D4248639910509F052C280919805CF5BDE4F4DC00E94432559
S12318408530D0F6FBCF0E94D424C82FD0E00E94D424C817D90709F03EC20E94D4248C0185
S123186090939905809398050E94D4240817190709F031C20E94D4248839910509F02BC257
S123188080919805CF51DE4F26C00E9443258530D0F6FBCF0E94D424C82FD0E00E94D42439
S12318A0C817D90709F017C20E94D4248C0190939905809398050E94D4240817190709F029
S12318C00AC20E94D4248F3A910509F004C280919805CF57DD4F8883FEC10E9443258530F7
S12318E0C8F6FBCFC0E0D0E00E944325823080F10E94D4240E94D4248F38910509F0EBC1A9
S123190010929905109298051CC0EF57FD4F108180E70E94F72482E00E94F7248091980554
S12319200E94F724812F0E94F7248FE80E94F724809198059091990501969093990580936D
S12319409805E0919805F0919905E03AF105E8F221965AEFC030D50709F4BDC1C5CF0E9452
S1231960D4248C010E94D424F82EEE24E00EF11E0E94D4248C0190939905809398050E94D5
S1231980D4240817190709F0A6C10E94D424883A9105A9F4D7010E944826E0708091980537
S12319A090919905E82BF92BF0939905E0939805D7010F010E94592612BC11BC8CC1E0919A
S12319C09605F091970509950E944325853038F6FBCFCC24DD240E944325833040F10E9475
S12319E0D424EC010E94D4248C010E94D4248D3A910509F070C1102F00270C0F1D1FD80120
S1231A000E944026F02C84E50E94F72483E00E94F7248F2D0E94F724802F0E94F724012F43
S1231A201127802F0E94F7248BEA0E94F7240894C11CD11C80E0C8168AEFD80609F44BC1C8
S1231A40CACFCC24DD240E9443258330C0F10E94D424EC010E94D4247C010E94D4248A3A8E
S1231A60910509F038C1FE2CEE24EC0EFD1ED7010E944026802D90E0D70111960E94402605
S1231A80002D10E0102F0027080F191F85E50E94F72484E00E94F724802F0E94F724012F8C
S1231AA01127802F0E94F7248E2D0E94F724EF2CFF248E2D0E94F7248AEA0E94F724089483
S1231AC0C11CD11C40E0C4164AEFD40609F403C1BACFC0E0D0E00E944325882359F00E94F1
S1231AE0D424873A910509F0F6C0E0919605F0919705099521965AEFC030D50709F4EBC0A9
S1231B00EACFC0E0D0E00E944325882369F00E94D4248039910509F0DEC00E94FD00E0911A
S1231B209605F0919705099521968AEFC030D80709F4D1C0E8CFC0E0D0E00E944325882302
S1231B40B1F00E94D424873D910509F0C4C080912A0590912B05ADE6B1E0082E0E944D266F
S1231B6012BC11BCE0919605F0919705099521964AEFC030D40709F4AEC0DFCFC0E0D0E0DB
S1231B800E9443258823B1F00E94D424863D910509F0A1C080912A0590912B05AEE6B1E0E8
S1231BA0082E0E944D2612BC11BCE0919605F0919705099521965AEFC030D50709F48BC060
S1231BC0DFCFC0E0D0E00E944325823010F10E94D424892B09F07FC00E94D42486389105D2
S1231BE0C1F489E70E94F72485E00E94F7248FEC0E94F7248FE30E94F7248CE00E94F7244D
S1231C0081E70E94F7248BE00E94F72486E80E94F72421968AEFC030D80709F45CC0D3CF8E
S1231C20C0E0D0E00E944325823008F44CC00E94D424892B09F047C00E94D4248C3A910548
S1231C4009F049C083E50E94F72488E00E94F72480913B0690913C060E94F72480913B0670
S1231C6090913C06892F99270E94F7248091FB059091FC050E94F7248091FB059091FC05A5
S1231C80892F99270E94F72480912B0690912C060E94F72480912B0690912C06892F9927AC
S1231CA00E94F72480912E0690912F060E94F72480912E0690912F06892F99270E94F7243B
S1231CC08CEA0E94F72421964AEFC030D40719F0A9CF0E94F724A895DF91CF911F910F9177
S1231CE0FF90EF90DF90CF9008950F931F93CF93DF93109200061092FF050E9440243C9A15
S1231D003D9A3F9A3E9A449A459A479A469A38984098399841983A9842983B98439838983D
S1231D2039983A983B9854985C9855985D9854985598239A249A259A2B9A2C982D98279A45
S1231D40269A5398529822985698219820980E944B24AAE5B1E00E944026802D80938B0548
S1231D600E945C1E0E94AE1E0E942E240E941C060E9477042B9A2C98A7E0B0E00E94402658
S1231D80802D12BC11BC85FF9BC080910001909101019F7D90930101809300010E94730376
S1231DA00E94C0030E94C1000E9486000E94FD0086E0AAE0B0E0082E0E944D2689E1ABE0D0
S1231DC0B0E0082E0E944D268EE1ACE0B0E0082E0E944D26AEE0B0E0082E0E944D2620E0E5
S1231DE030E0F901EF5DFC4F8081D901A25ABE4F082E0E944D262F5F3F4F2A30310589F7E3
S1231E0080912501A9E6B1E0082E0E944D2680912601AAE6B1E0082E0E944D26809127013F
S1231E20ABE6B1E0082E0E944D2680912801ACE6B1E0082E0E944D2620E030E0F901E0534C
S1231E40FA4F8081D901AE58BE4F082E0E944D262F5F3F4F2A30310589F720E030E0F901C6
S1231E60E053FA4F8089D901A458BE4F082E0E944D262F5F3F4F2A30310589F78091F30576
S1231E80A1E7B1E0082E0E944D26809114019091150166E070E00E94DC25ADE0B0E0062EF3
S1231EA00E944D2684E1ADE6B1E0082E0E944D2681EEAEE6B1E0082E0E944D2612BC11BCBB
S1231EC00E94E8000E9411010E949A000E946100809100019091010185FD07C080916F0083
S1231EE08B7F80936F00449A459A809124011092900510921D0580911401909115018D5D1D
S1231F00954030F08CED95E0909315018093140110927A0586B3866086BB78948AEA0E94D6
S1231F20F72480E00E94F72485E50E94F72489B1829586958695817080938D0580916E00A2
S1231F40836080936E002B9A2C9AA89580917D0590917E058E37910570F180917A05882323
S1231F6051F58091FF05909100069F7E909300068093FF0580916F00856080936F00809186
S1231F806E00836080936E002B9A81E080937A058091FF0590910006806290930006809359
S1231FA0FF058091FF05909100069062909300068093FF0547C080917A05813009F042C068
S1231FC080917D0590917E058E379105D8F580916F008D7F80936F00809170008C7F8093F1
S1231FE0700080916F008B7F80936F0080916E00836080936E008091FF05909100068F7D36
S1232000909300068093FF058091FF0590910006877F909300068093FF05389839983A9887
S12320203B9854985598449A459A10927A058091FF05909100069F7D909300068093FF057A
S12320401092780580917A058130F9F4809178058823C1F080916F00826080936F00809150
S1232060700083608093700080916E00836080936E008091FF059091000688609093000656
S12320808093FF052B9A2C9A13C010927805449A459A109278051092B300109284051092AA
S12320A0830580913F0190914001892B09F42B9840917D0550917E05209120013091210101
S12320C0809100019091010180709074822B932B4817590788F48091FF059091000697FD5D
S12320E00BC08091FF05909100069F7B909300068093FF05469A0AC08091FF059091000695
S12321009064909300068093FF054698F89480918505909186058A5A9A4AC1F080918505C2
S1232120909186058555954589F078948091FF05909100068064909300068093FF0588EEE0
S123214093E090933501809334010AC078948091FF05909100068F7B909300068093FF050B
S1232160F89480918705909188058A5A9A4AC1F080918705909188058555954589F0789487
S12321808091FF05909100068068909300068093FF0588EE93E090933501809334010AC083
S12321A078948091FF05909100068F77909300068093FF0580913401909135010B9758F006
S12321C02D9A80913401909135010197909335018093340101C02D9880911D05833009F4F5
S12321E003C1843018F4882371F08BC0853009F437C2853008F462C1863009F4EFC1873067
S123220009F0E6C275C280917B0590917C058D52914008F4E0C2E0911D05F0E08091780075
S1232220909179008C7F65E070E00E94DC25EE0FFF1FE65AFA4F7183608380911D05C82F18
S1232240D0E0E0911D05F0E0EE0FFF1FE25EFA4F80819181E0911D05F0E0EE0FFF1FE65AF2
S1232260FA4F20813181880F991F880F991F820F931F880F991F6AE070E00E94DC25CC0F76
S1232280DD1FC25EDA4F7983688310927C0510927B0580911D058F5F80931D0580911D0540
S12322A080937C000E94EB0880911E0590911F058A35910564F42091140130911501C90169
S12322C0880F991F820F931F9695879504C08091140190911501909317018093160180918A
S12322E03F0190914001892B09F470C280913F019091400101979093400180933F012B9A8E
S123230065C280917B0590917C058D52914008F462C290911D0540919505842F8370845067
S1232320990F990F980FE92FF0E0EE0FFF1FEE5FFE4F808191812091780030917900820FFE
S1232340931F969587959183808310927C0510927B05A89580911D05C42FD0E08130D1F49B
S12323608E01085F1F4F842F0E942D06000F111F025E1A4FF80191838083809195058823FF
S1232380A9F480912E0590912F050E949306809325060CC08081918162E070E00E94F02562
S12323A0CC0FDD1FCA5CDA4F7983688380911D058F5F80931D0580911D0580937C008091E3
S12323C02E0590912F058D38910514F082E309C080912E0590912F05893791050CF4FBC139
S12323E089E180937905F7C180917B0590917C058D52914008F4EFC1E0911D05F0E0809123
S12324007800909179009695879596958795EE0FFF1FE65AFA4F9183808380911D05C82F33
S1232420D0E0E0911D05F0E0EE0FFF1FE25EFA4F80819181E0911D05F0E0EE0FFF1FE65A10
S1232440FA4F20813181880F991F880F991F820F931F65E070E00E94DC25CC0FDD1FC25ECC
S1232460DA4F7983688310927C0510927B0580911D058F5F80931D0580911D0580937C00EB
S12324800E94EB08A895809195058F5F80939505843010F01092950590919505292F279561
S12324A02227279585B18F77822B85B99295990F907485B18F7B892B85B98DC180917B0508
S12324C090917C058159914008F485C180912401882331F1E0911D05F0E080917800909159
S12324E07900969587959695879590E0EE0FFF1FE65AFA4F91838083A0911D05B0E0E09152
S12325001D05F0E0EE0FFF1FE65AFA4F80819181AA0FBB1FA25EBA4F11969C938E933EC07D
S1232520E0911D05F0E08091780090917900EE0FFF1FE65AFA4F9183808380911D05C82F2C
S1232540D0E0E0911D05F0E0EE0FFF1FE25EFA4F00811181E0911D05F0E0EE0FFF1FE65AEF
S1232560FA4F808191810E9431079C01220F331F280F391FC80143E0880F991F4A95E1F780
S1232580801B910B820F931F6AE070E00E94DC25CC0FDD1FC25EDA4F7983688310927C0556
S12325A010927B0580911D058F5F80931D0580911D0580937C0020918D0589B1829586952E
S12325C08695817030E090E02817390709F4FEC0E0919605F09197050995F8C080917B0521
S12325E090917C058D52914008F4F5C0E0911D05F0E08091780090917900969587959695DC
S12326008795EE0FFF1FE65AFA4F9183808380911D05C82FD0E0E0911D05F0E0EE0FFF1F87
S1232620E25EFA4F80819181E0911D05F0E0EE0FFF1FE65AFA4F20813181880F991F880FBA
S1232640991F820F931F880F991F6AE070E00E94DC25CC0FDD1FC25EDA4F798368833EC0EA
S123266080917B0590917C058D52914008F4B3C0E0911D05F0E08091780090917900969553
S1232680879596958795EE0FFF1FE65AFA4F91838083E0911D05F0E0EE0FFF1FE65AFA4F11
S12326A02081318184E190E0FC012E9FC0012F9F900D3E9F900D11240E94D7069093290579
S12326C080932805809128059091290562E070E00E94F025709329056093280510927C056C
S12326E010927B0580911D058F5F80931D0568C080917B0590917C058D52914008F46BC02C
S1232700E0911D05F0E08091780090917900969587959695879590E0EE0FFF1FE65AFA4F8D
S1232720918380838091680590916905893791050CF1A0911D05B0E0E0911D05F0E0EE0FDB
S1232740FF1FE25EFA4F40815181E0911D05F0E0EE0FFF1FE65AFA4F20813181CA01880F7F
S1232760991F840F951F820F931F969587959695879519C0A0911D05B0E0E0911D05F0E066
S1232780EE0FFF1FE25EFA4F20813181E0911D05F0E0EE0FFF1FE65AFA4F80819181820F93
S12327A0931F96958795AA0FBB1FA25EBA4F11969C938E9310927C0510927B0510921D0580
S12327C080911D0580937C000E94EB08A89503C081E080931D0580917B0590917C0501963E
S12327E090937C0580937B050E949D0780917D0590917E058F55914008F457C0809123061F
S12328008F5F809323069091230680912406981708F44EC01092230680912C0590912D05EC
S1232820E0913406FF27E7FDF095EF5FF94F208130E08217930734F4809121069091220637
S1232840890F17C080912C0590912D05E0913406FF27E7FDF095EF5FF94F208130E0821756
S123286093074CF08091210682302CF08091210681508093210680912106E0913406FF272C
S1232880E7FDF095EF5FF94F2089992787FD909530E02817390764F4E0913406FF27E7FD87
S12328A0F095EF5FF94F808901C081E08093210680917D0590917E058739910508F461C0EA
S12328C020912A0530912B058091220190E04996281739070CF055C08091C5059091C60549
S12328E001969093C6058093C5052091C5053091C6058091C7059091C8052817390708F425
S123290042C01092C6051092C50520917D0530917E058091BF059091C0052817390730F403
S12329209091C3058091C405890F15C020917D0530917E058091BF059091C00549968217B9
S1232940930758F49091C3058091C205891728F48091C30581508093C3059091C305809191
S1232960C105891718F48091C10508C09091C3058091C205981738F48091C2058093C305F3
S123298002C01092C30580911C0582FF1BC080917D0590917E05805D9740A0F420912A051A
S12329A030912B058091220190E00596281739074CF481E080938F058091FF0590910006E0
S12329C0916007C010928F058091FF05909100069E7F909300068093FF0580910001909139
S12329E0010192FF27C020917D0530917E0580912E0190912F0182179307E0F420917D0517
S1232A0030917E0580913001909131012817390788F420912A0530912B058091220190E069
S1232A2005962817390734F48091FF0590910006946005C08091FF05909100069B7F9093E2
S1232A4000068093FF05809100019091010193FF37C04A9B35C020917D0530917E05809135
S1232A603201909133018217930730F48091FF0590910006986005C08091FF05909100063E
S1232A80977F909300068093FF0580911C0583FF0DC080917D0590917E05875D964030F04A
S1232AA08091CB059091CC05886005C08091CB059091CC05877F9093CC058093CB053DC0E5
S1232AC08091CB059091CC05877F9093CC058093CB058091370120912C0530912D0590E0B4
S1232AE08217930724F4809137018823B9F440917D0550917E0520911C0130911D01809171
S1232B0000019091010180709078822B932B8417950750F480911C0580FF06C08091FF0523
S1232B2090910006986005C08091FF0590910006977F909300068093FF05809100019091E8
S1232B40010180FF67C080912B0180FF11C08091B805883C28F08091C3058823B9F418C089
S1232B609091C3058091B8058695891790F010C080912B0182FF0DC08091B805883C48F03A
S1232B808091FF059091000696FF02C0549A01C0549880912B0184FF16C08091B805883CDB
S1232BA028F08091210618165CF12CC0209121068091B805332727FD3095869590E082174D
S1232BC093070CF11FC080912B0186FF1CC08091B805883CC0F020917D0530917E05809113
S1232BE02C0190912D018217930760F420912C0530912D0580918C0590E08217930714F4AC
S1232C00559A01C055988091B805883C28F01092B80502C0549855988091B8058F5F8093A0
S1232C20B80592C91F920F920FB60F9211248F939F93809135068F5F809335068091350663
S1232C40882309F446C08091FF05909100069061909300068093FF0510927A058091FF051F
S1232C60909100069F7D909300068093FF0580916F008B7F80936F0080916F008D7F809322
S1232C806F00809170008C7F8093700080916E00836080936E00449A459A8091FF059091DC
S1232CA000068F7D909300068093FF058091FF0590910006877F909300068093FF0538986C
S1232CC039983A983B985498559810927E0510927D0578949F918F910F900FBE0F901F9042
S1232CE01895282F8091FF059091000693FD08C0223019F0203221F402C04498089545985E
S1232D0008951F920F920FB60F9211248F9380912A01813019F482E08093CF058F910F9001
S1232D200FBE0F901F9018951F938091B105882309F466C02091B1058091B105823089F423
S1232D40449A8091870590918805880F991F9093880580938705809187059091880581607C
S1232D600BC08091B105803269F4459A8091870590918805880F991F9093880580938705E6
S1232D801092B10580918400909185009093BC058093BB05479A8091F6059091F705892B27
S1232DA061F080913006882341F08091F6059091F70590938B0080938A0080917D05909173
S1232DC07E058C5D954008F055C080911C0581FF51C080918A0090918B0088539F4F9093AB
S1232DE08B0080938A002093300680918A0090918B008C509E4F90932F0680932E063AC015
S1232E00809130068823B1F1109130061230A1F4809130060E9471168091850590918605B5
S1232E20880F991F9093860580938505809185059091860581600EC010913006103281F470
S1232E40809130060E9471168091850590918605880F991F90938605809385051093B105C4
S1232E6080912E0690912F0690938B0080938A00109230061F9108951F920F920FB60F928B
S1232E8011242F933F934F935F936F937F938F939F93AF93BF93EF93FF930E9494162B9A70
S1232EA07894FF91EF91BF91AF919F918F917F916F915F914F913F912F910F900FBE0F9097
S1232EC01F9018951F920F920FB60F9211242F938F939F93F8949091130190952091CF0524
S1232EE0243009F1253040F4223021F12330A8F4213009F06CC009C02731E1F1233609F4E5
S1232F0051C02E3009F063C01BC09093B20084E08093B100389A83E064C096BD83E085BDF9
S1232F203A9A84E05EC09093B2002093B1003B9A82E057C096BD83E085BD399A81E051C073
S1232F4081E0809306059093B20084E08093B1008091830590918405892B11F0389A3B9A52
S1232F6080918400909185009093BA058093B90587E137C081E08093070596BD83E085BD88
S1232F808091830590918405892B11F0399A3A9A80918400909185009093BE058093BD0598
S1232FA08EE01FC081E0809306059093B20084E08093B1008091830590918405892B21F03C
S1232FC0389A3B9A3A9A399A2093CF050CC09093B20084E08093B100389A3B9A3A9A399A01
S1232FE083E68093CF0578949F918F912F910F900FBE0F901F901895CF93DF93EC01809128
S12330008A05E7E0F0E0E81BF109EE0FFF1FE25EFA4F8081918120918905821B282F30E08F
S12330208091290190E0880F991F880F991FAC01429FC001439F900D529F900D112464E668
S123304070E00E94DC256436710520F083E68093310602C060933106809131066AE00E9486
S1233060D02580932806809128068A301CF089E08093280680917D0590917E05885E934077
S123308008F0B3C0109226068FEF8093340680912806992787FD909564E0880F991F6A95EE
S12330A0E1F78093810580917D0590917E0564E670E00E94DC25655060932D0680917D05B9
S12330C090917E05845F914060F410922D06E0912D06FF27E7FDF095E65CFE4F808190E038
S12330E0A3C080912D068430D9F5E0918105F0E0EF5BFE4F2081E0912D06FF27E7FDF09571
S1233100E65CFE4F6081E0912D06FF27E7FDF095E65CFE4F808190E09093CE058093CD052D
S1233120E091CD05F091CE0580917D0590917E0540912D0630E0220F331F261B3109845FC8
S123314091406CE94602A0011124840F951FAC01249FC001259F900D349F900D11243AC0AF
S1233160E0912D06FF27E7FDF095E55CFE4F6081E0912D06FF27E7FDF095E65CFE4F408126
S1233180E0912D06FF27E7FDF095E65CFE4F808190E09093CE058093CD05E091CD05F09159
S12331A0CE0580917D0590917E0520912D0670E0641B7109845F91404CE9240290011124FF
S12331C0820F931F9C01629FC001639F900D729F900D112464E670E00E94F025E60FF71F6B
S12331E0F093CE05E093CD05C7C080917D0590917E05875F9242E8F086E9809326068FE0C3
S12332008093340680912806909134068295807F890F80938105E0918105F0E0EF5BFE4F1E
S1233220808190E0880F991F9093CE058093CD05A3C080917D0590917E05885E934062E357
S123324070E00E94DC2560932606809126066AE00E94D02580933406809128069091340653
S12332608295807F890F80938105E0918105F0E0EF5BFE4F808190E0880F991F9093CE05EF
S12332808093CD058091340687FD39C0809134068F30ACF5E0918105F0E0EE5BFE4F808174
S12332A0E0918105F0E0EF5BFE4F6081E091CD05F091CE052091260640913406861B880F14
S12332C0992787FD909530E06AE04602A0011124241B350BAC01429FC001439F900D529FCB
S12332E0900D11246AE070E00E94F025772767FD70956E0F7F1F7093CE056093CD058091D9
S1233300280687FD39C0809128068930ACF5E0918105F0E0EF5AFE4F8081E0918105F0E040
S1233320EF5BFE4F6081E091CD05F091CE052091310640912806861B880F992787FD9095F2
S123334030E06AE04602A0011124241B350BAC01429FC001439F900D529F900D11246AE097
S123336070E00E94F025772767FD70956E0F7F1F7093CE056093CD0580917D0590917E054E
S1233380855F914010F46AEB66C080917D0590917E058952934210F06DE05DC080917D0511
S12333A090917E0585569941B0F080917D0590917E05845699416AE070E00E94DC25CB011C
S12333C0880F991F880F991F860F971F64E670E00E94DC2540C080917D0590917E05815AB1
S12333E09F40B0F080917D0590917E05805A9F406AE070E00E94DC25CB01E3E0880F991F3F
S1233400EA95E1F764E670E00E94DC25645123C080917D0590917E05855F914010F460E04C
S12334201AC080917D0590917E05845F91406AE070E00E94DC25CB019B0173E0220F331F48
S12334407A95E1F7880F991F820F931F64E670E00E94DC2567532091CD053091CE05862F2C
S1233460992787FD9095820F931F97FF06C08091CD059091CE0561E0681B20919B052456DA
S123348025310CF024E14091CD055091CE05809112019091790540585040480F511D491B66
S12334A05109822F2C3E0CF48CEE282F332727FD3095240F351F862F992787FD9095280FA3
S12334C0391F2A3031052CF46EE472E080E090E013C081E0253F38072CF064E670E080E07F
S12334E090E00AC088E592E0821B930B9C01B901882777FD8095982F20917F0530918005A3
S12335002C0F3D1F40E050E00E94B12528E037E040E050E00E940326DA01C901DF91CF9199
S12335200895AF92BF92CF92DF92EF92FF920F931F93CF93DF93EC01E0913406FF27E7FDAA
S1233540F095EF50FB4F808190E09093F5058093F4056091B5057091B605209113012695D8
S12335602695620F711D7695679580E090E02AE530E040E050E00E94B12520917F053091D9
S123358080052C0F3D1F13E0369527951A95E1F740E050E00E94032659016A01E09134067F
S12335A0FF27E7FDF095EF50FB4F808190E0B4EBEB2EF12CCC9664EB70E00E94F025E81AEF
S12335C0F90A0027F7FC0095102FEA0CFB1C0C1D1D1D9E0140E050E0C801B7010E94B1259E
S12335E022E130E040E050E00E940326CA01B9012AE030E040E050E00E9403262A97CE014F
S1233600A0E0B0E02A9682179307A407B50718F48AE090E003C0CE01821B930BDF91CF91B9
S12336201F910F91FF90EF90DF90CF90BF90AF9008950F931F93CF93DF9380918400909151
S1233640850090933A06809339068091840090918500C29708F404C380913506882349F0A5
S123366088EE9DEF90930505809304051092350666C0E0918400F0918500C0910405D09142
S123368005059E0136952795CE016AE070E00E94DC25261B370BE217F307A8F481E0809364
S12336A03806809184009091850090933C0680933B0680912A01823009F0D2C28091F00454
S12336C08093CF05CDC2809184009091850090932C0680932B06E0917F05F09180052091F0
S12336E08400309185008091EF0490E02C1B3D0BAC01429FC001439F900D529F900D112468
S12337006EE170E00E94F025CB018E0F9F1F62E070E00E94F0257093800560937F0510923E
S1233720800510927F058091840090918500909305058093040510928500109284008091F8
S12337407805893628F4809178058F5F80937805479880917D0590917E05C0910405D09130
S12337600505D093FC05C093FB052091FB053091FC05009101051091020540E050E060E042
S123378070E489E191E00E942526CA01B9012EE130E040E050E00E94B12520EC30E0A901D7
S12337A0049F9001059F300D149F300D11242050324040E050E00E94032630937E052093D5
S12337C07D052091A8053091A9054091A6055091A705C901880F991F820F931F840F951FEA
S12337E096958795969587959093A9058093A8058091A4059091A5059093A7058093A60594
S12338008091A2059091A3059093A5058093A4058091A0059091A1059093A3058093A20598
S123382080919E0590919F059093A1058093A00580919C0590919D0590939F0580939E0598
S123384080917D0590917E0590939D0580939C0580917D0590917E058D5D9540D8F0409125
S12338609B0580919C0590919D052091A8053091A905821B930B23E0429FA0011124840FDA
S1233880951F64E0969587956A95E1F78B5A80939B050FC084E680939B0580917F059091D4
S12338A0800564E070E00E94F0257093800560937F051092350680917D0590917E05805948
S12338C0914060F58091010590910205049731F180913806813011F584E090E090930205BE
S12338E08093010580910105909102058068809381001092850010928400D695C795D69571
S1233900C795D0930505C09304058091FB059091FC05969587959695879532C080917D0538
S123392090917E058955924078F18091010590910205039749F180913806813029F583E032
S123394090E0909302058093010580910105909102058068809381001092850010928400A8
S1233960CC0FDD1FCC0FDD1FD0930505C09304058091FB059091FC05880F991F880F991FFB
S12339809093FC058093FB058091FB059091FC050E94FC1790932F0680932E068091CB0584
S12339A09091CC0583FF39C0C091B205D091B305CE0163E070E00E94DC25892B41F1809179
S12339C0FB059091FC0563E070E00E94DC2570932F0660932E06E0912E06F0912F06209120
S12339E038018091FB059091FC0568E270E00E94DC2530E0629FC001639F900D729F900DFB
S1233A0011248E0F9F1F90932F0680932E062196D093B305C093B20504C01092B3051092D7
S1233A20B20580917D0590917E058A58924018F484E690E009C080911E0590911F058E36F4
S1233A4091053CF488EC90E0909337068093360604C0109237061092360680912E06909122
S1233A602F0620911601309117014091360650913706821B930B841B950B90932A06809361
S1233A8029068091290690912A0697FF20C08091290690912A062091FB053091FC05409117
S1233AA02E0650912F06820F931F8417950778F42091FB053091FC0580912E0690912F06C4
S1233AC0821B930B449690932A0680932906F89480917D0590917E05805E9E4208F095C06A
S1233AE08091FF059091000693FD8FC08091290690912A068739910504F11092B105809162
S1233B00290690912A0690938B0080938A0080918A0090918B009093F7058093F605809151
S1233B203806882311F480E201C082E0809330061092B10584E090E05CC08091290690911C
S1233B402A068B5B9F4F2CF11092B10584E690E090938B0080938A009093F7058093F60596
S1233B6080913806882311F480E201C082E080933006809130060E9471161092B10588E242
S1233B8090E09093F9058093F80584E18093030534C080912E0690912F0690938B008093B0
S1233BA08A002091FB053091FC058091290690912A06820F931F9093F7058093F6058091F2
S1233BC03806882341F480E20E94711680E28093B10582E007C082E00E94711682E08093E4
S1233BE0B10580E28093300684E18093030584EB90E09093F9058093F805109238068091DF
S1233C00FF05909100069F770FC08091FB059091FC058C509E4F90938B0080938A00809138
S1233C20FF05909100069068909300068093FF0580917D0590917E058D549D4138F08091EE
S1233C408400909185008C599F4F06C08091FB059091FC050E94911A9093890080938800D6
S1233C607894DF91CF911F910F9108951F920F920FB60F9211242F933F934F935F936F9320
S1233C807F938F939F93AF93BF93EF93FF930E94191B2B9A7894FF91EF91BF91AF919F919B
S1233CA08F917F916F915F914F913F912F910F900FBE0F901F9018951092800081EF9FEFE9
S1233CC0909389008093880085EF9FEF90938B0080938A00109285001092840084E090E02B
S1233CE09093020580930105809101059091020580688093810080916F00876080936F00D9
S1233D00539852983C9A3D9A449A459AA2E0B2E00E944026802D8093EF04A1E0B2E00E94DC
S1233D204026802D8093F0048091F0048E3039F08091F004873119F087E18093F004809133
S1233D408B05813021F4809169008C6003C080916900886080936900E99A089521EB30E0C6
S1233D60F90110821092B6001092B2001092B300A0E7B0E08C9183608C9338984098399803
S1233D8041983A9842983B984398389839983A983B98EFE6F0E080818D7F80838C918C7FC9
S1233DA08C9386E0F901808384E68093F0050895813099F438983B9880912A01843021F488
S1233DC039983A98109207051092400610923F06109206051092B1000895823049F4399862
S1233DE03A9810923E0610923D061092070515BC08951F920F920FB60F9211242F933F9385
S1233E004F935F936F937F938F939F93AF93BF93EF93FF93F89480910605843051F4809108
S1233E20B20090E09093FE058093FD0581E00E94D81E7894FF91EF91BF91AF919F918F912C
S1233E407F916F915F914F913F912F910F900FBE0F901F9018950F931F9380911E059091DE
S1233E601F050A9714F487E003C080918F0586E08093B1001092B20080917D0590917E05ED
S1233E80845F914018F410922D0616C080917D0590917E058D56974020F08EE080932D06FE
S1233EA00BC080917D0590917E0564E670E00E94DC25655060932D06E0912D06F0E0E55D2E
S1233EC0FC4F80818093130180918F05882329F02091F1018091180108C0E0918105F0E0A6
S1233EE0EF51FE4F808120911801829FC00111249093B6058093B50580917D0590917E056D
S1233F008059914048F5809100019091010182FF19C08091B5059091B60520911901820F24
S1233F20911D9093B6058093B5058091FF05909100068460909300068093FF058EE1809342
S1233F40B4053FC08091FF05909100068B7F909300068093FF0535C08091FF0590910006EE
S1233F608B7F909300068093FF058091B405823028F08091B40581508093B405E091B505CD
S1233F80F091B60580911901209119014091B405E80FF11D8EE190E0841B910930E0AC0187
S1233FA0429FC001439F900D529F900D11246EE170E00E94DC25E61BF70BF093B605E09323
S1233FC0B50580918F05882309F0ABC1E0918105F0E0EF51FE4F808120911801829FC0016D
S1233FE011249093B6058093B5058091340687FD3EC0809134068F30D4F5E0918105F0E076
S1234000EE51FE4F6081E0918105F0E0EF51FE4F40810091B5051091B60580912606209185
S12340203406E091180170E0641B710990E04AE0240290011124821B930B9C01629FC0014F
S1234040639F900D729F900D11246AE070E00E94F025F0E06E9FC0016F9F900D7E9F900D86
S12340601124800F911F9093B6058093B5058091280687FD3EC0809128068930D4F5E0912A
S12340808105F0E0EF50FE4F6081E0918105F0E0EF51FE4F40810091B5051091B60580918C
S12340A0310620912806E091180170E0641B710990E04AE0240290011124821B930BAC01A5
S12340C0649FC001659F900D749F900D11246AE070E00E94F025F0E06E9FC0016F9F900DF8
S12340E07E9F900D1124800F911F9093B6058093B505809100019091010184FF55C0209165
S123410048053091490580912A0590912B0528173907C4F480912A0590912B0520914805E8
S123412030914905821B930B64E070E00E94F02580918205861710F46093820580912301FE
S12341408093B7053091B7053430C8F08091B5059091B605E0918205F0E0EF5DFC4F20814C
S1234160820F911D9093B6058093B50531503093B7058091FF0590910006806109C01092C9
S123418082051092B7058091FF05909100068F7E909300068093FF0580912A0590912B051C
S12341A09093490580934805809100019091010191FFB4C080918D05882309F0AFC080912A
S12341C0F2058F5F8093F2059091F2058091F305981708F4A6C01092F205809126059091C4
S12341E02705E0912806FF27E7FDF095E053FA4F208130E028173907B4F4809126059091B0
S12342002705E0912806FF27E7FDF095E053FA4F2081821B910962E070E00E94F0256C59DE
S12342206093F0052BC08091260590912705E0912806FF27E7FDF095E053FA4F208130E0C3
S123424082179307DCF48091F0051816BCF4E0912806FF27E7FDF095E053FA4F8081209117
S123426026053091270590E0821B930B62E070E00E94F02584E6861B8093F0058091FF0506
S1234280909100069D7F909300068093FF052091F005E0912806FF27E7FDF095E053FA4F47
S12342A08089332727FD309590E08C599F4F8217930754F4E0912806FF27E7FDF095E0538F
S12342C0FA4F80898C591EC02091F005E0912806FF27E7FDF095E053FA4F4089332727FD2E
S12342E0309584E690E0841B910928173907CCF4E0912806FF27E7FDF095E053FA4F9089E0
S123430084E6891B8093F0058091FF05909100069260909300068093FF0503C084E68093D5
S1234320F0058091B5059091B6052091250630E062E070E00E94F025269FC001279F900DBF
S1234340369F900D112464E670E00E94DC25660F771F7093B6056093B50520913405309154
S1234360350580911B0190E0C29628173907D4F5809100019091010181FF34C080913405CF
S123438090913505C397D4F040911A0180911A01209134053091350560911B0190E070E0D6
S12343A06E5C7F4FFC01E29FC001E39F900DF29F900D11240E94DC25461B03C080911A01AD
S12343C0482F50E08091B5059091B605480F591F5093B6054093B5058091FF059091000655
S12343E0826005C08091FF05909100068D7F909300068093FF0580912401882371F0209197
S1234400B5053091B6058091F00524563040992787FD9095280F391F0DC02091B505309181
S1234420B6058091F0052C593F4F992787FD9095281B390B3093B6052093B5058091CB05E8
S12344409091CC0583FF1CC0E091B505F091B605209139018091B5059091B60564E170E07A
S12344600E94F02530E0629FC001639F900D729F900D11248E0F9F1F9093B6058093B50527
S1234480809100019091010190FF4CC080911E0590911F05823891050CF044C08091B505B4
S12344A09091B60520912501820F911D9093B6058093B505E0911E05F0911F056091180118
S12344C02091250182E890E08E1B9F0B70E0AB01849FB001859F700D949F700D11248FEF00
S12344E090E0FB01E89FB001E99F700DF89F700D1124882777FD8095982F30E040E050E067
S12345000E94B12520E43FE140E050E00E9403268091B5059091B605820F931F9093B60518
S12345208093B5052091B5053091B6058091180145EF849FC00111248217930754F48091C0
S12345401801849FC00111249093B6058093B5050BC08091B5059091B6051816190624F0A7
S12345601092B6051092B5058091FF059091000692FF05C0109284051092830510C0209116
S12345808305309184058091B5059091B605820F931F9695879590938405809383054091FC
S12345A07D0550917E0520911C0130911D01809100019091010180709078822B932B48176D
S12345C0590730F48091FF05909100069F770DC080911C0580FD04C010928405109283056C
S12345E08091FF05909100069068909300068093FF0578941F910F9108951F920F920FB633
S12346000F9211242F933F934F935F936F937F938F939F93AF93BF93EF93FF93F89420910B
S12346200605223039F0243009F44FC0213009F051C01CC080913F06909140068F3F910538
S1234640D1F1C8F180913F06909140068F5F8093B30080913F06909140068F5F90409093CC
S1234660400680933F062093060534C00E942B1F80918305909184059093400680933F06F6
S123468080913F06909140068F3F9105A1F098F080913F06909140068F5F8093B30080915A
S12346A03F06909140068F5F90409093400680933F0682E007C080913F06909140068093D2
S12346C0B30084E08093060505C081E00E94D81E109206057894FF91EF91BF91AF919F915A
S12346E08F917F916F915F914F913F912F910F900FBE0F901F9018951F920F920FB60F9207
S123470011242F933F934F935F936F937F938F939F93AF93BF93EF93FF93F894209107059F
S1234720223039F0243009F453C0213009F053C020C080913D0690913E068F3F910591F0BB
S123474088F080913D0690913E068F5F87BD80913D0690913E068F5F904090933E06809301
S12347603D0633C080913D0690913E0687BD84E024C0809183059091840590933E068093FD
S12347803D0624E025BD16BC80913D0690913E068F3F9105A9F0A0F080913D0690913E061B
S12347A08F5F87BD80913D0690913E068F5F904090933E0680933D0682E0809307050BC043
S12347C080913D0690913E0687BD2093070503C082E00E94D81E7894FF91EF91BF91AF91B0
S12347E09F918F917F916F915F914F913F912F910F900FBE0F901F9018951F920F920FB677
S12348000F9211242F933F934F935F936F937F938F939F93AF93BF93EF93FF93F8948091A9
S12348200705843049F486B590E09093CA058093C90582E00E94D81E7894FF91EF91BF9193
S1234840AF919F918F917F916F915F914F913F912F910F900FBE0F901F90189554985C980D
S123486055985D985498559815BCEEE6F0E080818360808384E085BD16BC82E187BD089561
S123488011B88FEF84B915B887B98AB90895089508950895089588E98093C10083E1809373
S12348A0C40088E896E09093460680934506909342068093410688E496E090934406809356
S12348C043069093C9068093C806109247061092FA0508951F920F920FB60F9211248F937C
S12348E09F93EF93FF9380914706882311F1E0914506F091460681918093C600F093460620
S1234900E0934506E85CF64030F088E896E0909346068093450680914706815080934706F9
S123492080914706882329F48091C1008F7D8093C100FF91EF919F918F910F900FBE0F9030
S12349401F9018951F920F920FB60F9211242F938F939F93EF93FF938091C600E091C806CA
S1234960F091C90680838091FA058F5F8093FA058091C8069091C90601969093C906809365
S1234980C8068858964030F088E496E09093C9068093C806FF91EF919F918F912F910F90FB
S12349A00FBE0F901F9018958091FA05882319F48FEF9FEF0895F8948091FA05815080933A
S12349C0FA05E0914306F09144062191F0934406E0934306E858F64030F088E496E0909379
S12349E04406809343067894822F90E00895982F809147068F33E0F780914706803418F06B
S1234A0080E090E00895F894809147068F5F80934706E0914106F091420690838091410601
S1234A209091420601969093420680934106885C964030F088E896E0909342068093410628
S1234A408091C10080628093C100789481E090E00895CF93DF93EC0104C00E94F72481117C
S1234A60219688818823C9F781E090E0DF91CF91089588E095E00E942925089580E195E089
S1234A800E94292508958091FA0590E00895CF92DF92EF92FF920F931F93CF93DF93CDB7D8
S1234AA0DEB729970FB6F894DEBF0FBECDBF8C01F62EE42EDE011196E3E1F5E089E001907A
S1234AC00D928150E1F749E06E010894C11CD11CFF2081F089E090E0841B91092F2D30E07E
S1234AE08217930738F04150F601E40FF11D8CE28083FF244150F601E40FF11DC8016AE09E
S1234B0070E00E94DC25805D8083C8016AE070E00E94DC258B01672B11F4FF2019F085E008
S1234B208F15B0F619E01E197E010894E11CF11C07C0F701E10FF11D80810E94F7241F5FD9
S1234B401930B8F329960FB6F894DEBF0FBECDBFDF91CF911F910F91FF90EF90DF90CF905B
S1234B600895629FD001739FF001829FE00DF11D649FE00DF11D929FF00D839FF00D749F45
S1234B80F00D659FF00D9927729FB00DE11DF91F639FB00DE11DF91FBD01CF01112408953A
S1234BA0991B79E004C0991F961708F0961B881F7A95C9F780950895AA1BBB1B51E107C056
S1234BC0AA1FBB1FA617B70710F0A61BB70B881F991F5A95A9F780959095BC01CD010895E0
S1234BE097FB092E07260AD077FD04D0E5DF06D000201AF4709561957F4F0895F6F7909559
S1234C0081959F4F0895A1E21A2EAA1BBB1BFD010DC0AA1FBB1FEE1FFF1FA217B307E40792
S1234C20F50720F0A21BB30BE40BF50B661F771F881F991F1A9469F760957095809590953E
S1234C409B01AC01BD01CF01089597FB092E05260ED057FD04D0D7DF0AD0001C38F4509525
S1234C604095309521953F4F4F4F5F4F0895F6F790958095709561957F4F8F4F9F4F089510
S1234C80F999FECFB2BDA1BDF89A119600B40895F7DFE02DF5DFF02D0895F999FECFB2BD1B
S1234CA0A1BD00BC11960FB6F894FA9AF99A0FBE0895F3DF012CF1DF11240895FFCF2F00AF
S1234CC0010002000300040005000600070008003228E803900106141E3C401F401F641927
S1234CE0121E01010203040A0411C409C4098813AC0D6400DCE603020A143246965000546D
S1234D00819596B7AFC3C8BEBEB9B0AFAFADAC4984C0CBD2D6D7D0C7C2BBB8B3AEAAA945BA
S1234D208AA2A9AAB7C0BABEBBB6B8B2B3B4B93281868DA4A58B8C8F9EA6A2A6A5A6C03486
S1234D40525D5B596F788285858281FF859FB034444E4B4A54615769727272737D90952741
S1234D602C1B252B334B5155616A6D6C7D828B1D211A242A32454C4F5E6169717E8186343C
S1234D80323232323232323232327F323232323232323232323232323232323232323213A1
S1234DA01718191B1C1D1F21232527282C2E311418191A1C2124272B3035393C3E4143162D
S1234DC0191D232A31353B3F42484E565A5E651B1D363E525863666C6E777D84898D9322E5
S1234DE026434B6172818A9097A8ACAFB1B6B9292E484E6B7C939BA2AFB9BFCBD2D2D2299E
S1234E00344B536E7F9CA8B1BCC5D0D2D2D2D2283F4E587187A4B2BAC2D2D2D2D2D2D23747
S1234E2046545E7691B1BEC4D2D2D2D2D2D2D239485660869FBAD2D2D2D2D2D2D2D2D20006
S1234E4000000000000000000000000000000000000000000000000000000000000000004E
S1234E6000000000000000000000000000000000000000000000000000000000000000012D
S1234E8002030405060708090A0B0C0D0E0F100102030405060708090A0B0C0D0E0F1001FE
S1234EA002030405060708090A0B0C0D0E0F1014161718191A1B1C1D1E1F20212223241987
S1234EC01A1B1C1D1E1F2021222324252627271E1F2022232425262728292A2B2C2D2E007B
S1234EE00204060708090A0C0E28262422201E1E1E1E1E1E1E1E1E1E1EF0FF80BBE08804D2
S1234F0065484BA438022BF0207019CC13860F440CC209D0074C061B052A046A03D1025657
S1234F2002F201A1015F012801FB00D600B7009D0087007500660059004D0044003C00346C
S1234F40002E0029002500F0FF80BBE0880465484BA438022BF0207019CC13860F440CC21B
S1234F6009D0074C061B052A046A03D1025602F201A1015F012801FB00D600B7009D00874B
S1234F80007500660059004D0044003C0034002E0029002500F0FF80BBE0880465484BA42A
S1234FA038022BF0207019CC13860F440CC209D0074C061B052A046A03D1025602F201A1BD
S1234FC0015F012801FB00D600B7009D0087007500660059004D0044003C0034002E00290B
S1234FE0002500F0FF80BBE0880465484BA438022BF0207019CC13860F440CC209D0074CA6
S1235000061B052A046A03D1025602F201A1015F012801FB00D600B7009D008700750066FB
S12350200059004D0044003C0034002E00290025000000F5047E05AE066C08C00AB30D6305
S12350400F8B10D7118813000000000A000F001E003C007800FA007201E0018002800200E2
S12350600008000A000C000E00C80A4A067E0484031A002000270032003E0066008E00B25E
S123508002EB02240337034B03560361037003E800D600C200B0009D008A00780078006592
S12350A000520040002D0019000700000001175A5A5A5050505050505050505050505003D4
S11D50C0003200FA04041B5B481B5B324A000D0A00202020202020202020B7
S503028773
